 adcsdk

 Timestamp is 4fb04cb1 (Mon May 14 12:07:13 2012)

 Preferred load address is 10000000

 Start         Length     Name                   Class
 0001:00000000 00000004H .CRT$XCA                CODE
 0001:00000004 00000004H .CRT$XCZ                CODE
 0001:00000008 00000004H .CRT$XIA                CODE
 0001:0000000c 00000004H .CRT$XIZ                CODE
 0001:00000010 00000004H .CRT$XPA                CODE
 0001:00000014 00000004H .CRT$XPZ                CODE
 0001:00000018 00000004H .CRT$XTA                CODE
 0001:0000001c 00000004H .CRT$XTZ                CODE
 0001:00000020 0000003cH .rdata                  CODE
 0001:0000005c 00000023H .rdata$debug            CODE
 0001:00000080 00000674H .text                   CODE
 0001:000006f4 00000000H .xdata                  CODE
 0001:000006f4 00000014H .idata$2                CODE
 0001:00000708 00000014H .idata$3                CODE
 0001:0000071c 00000034H .idata$4                CODE
 0001:00000750 0000000cH .idata$6                CODE
 0001:00000760 0000008fH .edata                  CODE
 0002:00000000 00000034H .idata$5                DATA
 0002:00000034 0000003cH .data                   DATA
 0002:00000070 00000014H .bss                    DATA
 0003:00000000 00000058H .pdata                  DATA

  Address         Publics by Value              Rva+Base       Lib:Object

 0000:00000000       ___safe_se_handler_table   00000000     <absolute>
 0000:00000000       ___safe_se_handler_count   00000000     <absolute>
 0001:00000000       __xc_a                     10001000     corelib0:crt0init.obj
 0001:00000004       __xc_z                     10001004     corelib0:crt0init.obj
 0001:00000008       __xi_a                     10001008     corelib0:crt0init.obj
 0001:0000000c       __xi_z                     1000100c     corelib0:crt0init.obj
 0001:00000010       __xp_a                     10001010     corelib0:crt0init.obj
 0001:00000014       __xp_z                     10001014     corelib0:crt0init.obj
 0001:00000018       __xt_a                     10001018     corelib0:crt0init.obj
 0001:0000001c       __xt_z                     1000101c     corelib0:crt0init.obj
 0001:0000003c       ??_C@_1BE@FABCBOME@?$AAM?$AAU?$AAT?$AAE?$AAX?$AA_?$AAA?$AAD?$AAC?$AA?$AA@ 1000103c     adcsdk_common_topaz_v1:adc_sdk.obj
 0001:00000050       ??_C@_1M@EPBPGMBG@?$AAA?$AAD?$AAC?$AA1?$AA?3?$AA?$AA@ 10001050     adcsdk_common_topaz_v1:adc_sdk.obj
 0001:00000080       AdcInit                    10001080 f   adcsdk_common_topaz_v1:adc_sdk.obj
 0001:00000118       AdcDeinit                  10001118 f   adcsdk_common_topaz_v1:adc_sdk.obj
 0001:00000164       AdcConfigureChannel        10001164 f   adcsdk_common_topaz_v1:adc_sdk.obj
 0001:00000254       AdcGetSamples              10001254 f   adcsdk_common_topaz_v1:adc_sdk.obj
 0001:000003f8       DllEntry                   100013f8 f   adcsdk_common_topaz_v1:adc_sdk.obj
 0001:00000410       CloseHandle                10001410 f   coredll:COREDLL.dll
 0001:00000420       CreateMutexW               10001420 f   coredll:COREDLL.dll
 0001:00000430       CreateFileW                10001430 f   coredll:COREDLL.dll
 0001:00000440       ReleaseMutex               10001440 f   coredll:COREDLL.dll
 0001:00000450       DeviceIoControl            10001450 f   coredll:COREDLL.dll
 0001:00000460       WaitForSingleObject        10001460 f   coredll:COREDLL.dll
 0001:00000470       DisableThreadLibraryCalls  10001470 f   coredll:COREDLL.dll
 0001:00000480       _DllEntryCRTStartup        10001480 f   corelib0:pegdentry.obj
 0001:000005c4       _cexit                     100015c4 f   corelib0:cexit.obj
 0001:000005e0       _initterm                  100015e0 f   corelib0:crt0dat.obj
 0001:00000614       _cinit                     10001614 f   corelib0:crt0dat.obj
 0001:00000648       __security_init_cookie     10001648 f   corelib0:seccinit.obj
 0001:000006a4       free                       100016a4 f   corelib1:COREDLL.dll
 0001:000006b4       __security_gen_cookie2     100016b4 f   corelib1:COREDLL.dll
 0001:000006c4       DeleteCriticalSection      100016c4 f   coredll:COREDLL.dll
 0001:000006d4       InterlockedExchange        100016d4 f   coredll:COREDLL.dll
 0001:000006e4       TerminateProcess           100016e4 f   coredll:COREDLL.dll
 0001:000006f4       __IMPORT_DESCRIPTOR_COREDLL 100016f4     coredll:COREDLL.dll
 0001:00000708       __NULL_IMPORT_DESCRIPTOR   10001708     coredll:COREDLL.dll
 0002:00000000       __imp_CloseHandle          10002000     coredll:COREDLL.dll
 0002:00000004       __imp_CreateMutexW         10002004     coredll:COREDLL.dll
 0002:00000008       __imp_CreateFileW          10002008     coredll:COREDLL.dll
 0002:0000000c       __imp_ReleaseMutex         1000200c     coredll:COREDLL.dll
 0002:00000010       __imp_DeviceIoControl      10002010     coredll:COREDLL.dll
 0002:00000014       __imp_WaitForSingleObject  10002014     coredll:COREDLL.dll
 0002:00000018       __imp_DisableThreadLibraryCalls 10002018     coredll:COREDLL.dll
 0002:0000001c       __imp_free                 1000201c     corelib1:COREDLL.dll
 0002:00000020       __imp___security_gen_cookie2 10002020     corelib1:COREDLL.dll
 0002:00000024       __imp_DeleteCriticalSection 10002024     coredll:COREDLL.dll
 0002:00000028       __imp_InterlockedExchange  10002028     coredll:COREDLL.dll
 0002:0000002c       __imp_TerminateProcess     1000202c     coredll:COREDLL.dll
 0002:00000030       \177COREDLL_NULL_THUNK_DATA 10002030     coredll:COREDLL.dll
 0002:00000068       __security_cookie          10002068     corelib0:seccinit.obj
 0002:0000006c       __security_cookie_complement 1000206c     corelib0:seccinit.obj
 0002:00000074       _exitflag                  10002074     corelib0:cexit.obj
 0002:00000078       __onexitend                10002078     <common>
 0002:0000007c       __onexitbegin              1000207c     <common>
 0002:00000080       g_pcsExit                  10002080     <common>

 entry point at        0001:00000480

 Static symbols

 0001:000004c8       doexit                     100014c8 f   corelib0:cexit.obj
